:101A400017C01A3A4005930B0902120001010080E9
:101A50003209040000000000000012011001FF0024
:101A60000008D01653070102000000010403090416
:101A7000112420E0A0E6B0E001C01D92AC38B2070E
:101A8000E1F776C1A82FB92F80E090E041E050EA5D
:101A9000609530E009C02D9182279795879510F0C9
:101AA00084279527305EC8F36F5FA8F30895EADFB7
:101AB0008D939D930895CF93CFB7CF93DF93C39525
:101AC000B39BE9F7B39B0BC0B39B09C0B39B07C0A3
:101AD000B39B05C0B39B03C0B39B01C08FC06F9382
:101AE000C0916E00DD27CA58DF4F2F9365E5B39B89
:101AF00003C02F916F91E6CF0F931F934F9320E078
:101B000040E15F9306B3087103FB27F93F9350E070
:101B10003BE039C0187140642F77012F5F5F1EC012
:101B2000406816B318712F7752501FC0406406B337
:101B30002F770871D1F15F5F00C023C0406216B3F8
:101B40002F77187191F15F5F00C025C008711027D1
:101B5000515012F45D5F0000115027952C3F16B3D1
:101B6000C8F618710127015027952C3FC8F6422767
:101B7000499306B3087110274F73115027952C3FD6
:101B8000A8F64695469516B3187179F001270150CD
:101B900027952C3F98F66B5A60F3315006B3B0F698
:101BA00000C010E21ABF00271DC03B503195C31B77
:101BB000D04010E21ABF0881033C29F10B3419F11F
:101BC00020916C001981110F1213EDCF093651F1DC
:101BD0000D3211F0013E39F7CAE01AB715FD02C007
:101BE000CA95D9F7009374003F915F914F911F916F
:101BF0000F912F916F91CAB7C5FD61CFDF91CF9142
:101C0000CFBFCF91089520917400222369F31091E2
:101C10007200112309F534300AF1309372002093D9
:101C20006D001CC0009172000130B4F40AE53091DF
:101C30006F0034FD14C000936F00C1E6D0E013C004
:101C4000052710E000C0000008BB1AC0052710E0FF
:101C5000221F1DC010E021C04AE502C032ED432F13
:101C6000C4E1D0E032E017B31861C39A08B317BBE0
:101C700058E120E865E320FF052708BB2795179565
:101C80001C3FF0F66695B8F7B1F720FF052708BBB3
:101C9000279517951C3FD0F62795179517FF052711
:101CA00000001C3F08BBB0F629913A9519F7077E52
:101CB00010917300110FC651D04008BB11F0109362
:101CC0006C0010E21ABF086017B3177E402F477EE2
:101CD00054E05A95F1F708BB17BB48BB85CF2FEFEF
:101CE000B0E8A0E04BE0B1BF00008DE79CE0B39905
:101CF000FECFB39BFECF0197B399FDCF97FF03C0F3
:101D0000BA1B819501C0BA0FA69539F4A0E428F456
:101D1000281710F031B7282FA1E0415021F731BF2B
:101D200000000895F20121E00C0120935700E8958E
:101D30001124C20102962C01089514BE88E181BDD0
:101D400087E081BDBB9A2FEF85EA9EE0215080405D
:101D50009040E1F700C00000BB988AE580936F00D7
:101D60008FEF80936000AC9A8BB780628BBF089531
:101D7000E4DF712C312C412C512C14E6C5EDD4E15B
:101D800086B3887109F014E6115029F4109273009B
:101D900010926C00A4DF0AB605FE05C08CDE80E25E
:101DA0008ABF712C03C02197209751F7A89522E094
:101DB00032120CC0E0E4FAE1E054F10983E08093D0
:101DC0005700E8953097C1F7412C512C832D803472
:101DD00059F4F2013297E0348AE1F80750F485E0D3
:101DE00080935700E89505C0843019F4CD2B11F489
:101DF000E9C0312C80917200835087FD98C090918A
:101E00006D009D3209F091C0883009F08EC083ECDE
:101E1000809361008AE580936F00909177009076BF
:101E200080917800992361F1811108C082E49AE1E0
:101E3000909371008093700026E06CC0813059F45B
:101E40004114510409F44CC080917B00807C482EE1
:101E500050907C0045C0833081F48091790090914E
:101E60007A0060DF80917B0090917C005BDF842DA5
:101E70008F73B1F580E4382E33C08F73382E30C0A5
:101E80009091790010926A00811106C010926B0047
:101E90008AE690E022E03AC0853019F4909373000E
:101EA00027C08630F9F480917A00813019F48AE5F0
:101EB0009AE104C0823041F488E49AE19093710081
:101EC0008093700022E126C0833051F4911108C044
:101ED0008CE69AE1909371008093700024E01AC020
:101EE00020E018C0883079F0893031F49093750083
:101EF0008AE690E020E00AC021E08A3009F020E084
:101F00008AE690E003C085E790E021E090937100BD
:101F10008093700080917E00811105C080917D00CA
:101F2000821708F4282F209360001092720080918D
:101F30006F0084FF31C0809160008F3F69F1C82F2E
:101F4000893008F0C8E08C1B8093600080916100AC
:101F500098E8892780936100CC2391F0E09170008C
:101F6000F091710082E690E0DC0124912D9331968E
:101F70002C2F280F2A13F9CFF0937100E0937000F3
:101F80006C2F82E690E093DDCC5FCC3019F08FEFC0
:101F900080936000C0936F00C30101963C01803BB9
:101FA000944029F4EDE3FAE1E491EF3F59F40AB6E5
:101FB00005FEE3CE8CE1B39B8CE18150E1F780E23A
:0E1FC0008ABFDBCEBADE1BBE15BA38CDFFCF0E
:0400000300001A409F
:00000001FF
